:10000000F01F001055380000513800005138000032
:100010005138000051380000513800000000000045
:100020000000000000000000000000005138000047
:100030005138000000000000513800001116000087
:10004000E1130000E1130000E1130000E1130000E0
:10005000E1130000E1130000E1130000E1130000D0
:10006000E1130000E1130000E1130000E1130000C0
:10007000E11300004D3800004D3800004D380000FD
:10008000C9160000E1160000F91600001117000063
:100090004D380000D91700004D3800004D380000E1
:1000A0004D3800004D3800004D3800004D3800003C
:1000B0004D3800004D3800004D3800004D3800002C
:1000C00008B500230B60036000F00CFE08BD08B506
:1000D0000A20002101F098FA08BD000038B5094B4C
:1000E0000D1C041C1968012001F03EFB012001F0E9
:1000F0001BFB291C201C02F00DFF012001F024FB3A
:1001000038BDC046B004001070B5054E051C0E2465
:10011000013C295D301C01F081FD002CF8D170BD3F
:10012000843A000038B5164801F078FD154C201CC3
:10013000FFF7EAFF144D4221281C01F06FFD201C3F
:100140000E30FFF7E1FF4321281C01F067FD201C62
:100150001C30FFF7D9FF0D4801F060FD201C2A304C
:10016000FFF7D2FF281C4E2101F058FD201C38302B
:10017000FFF7CAFF616D064801F050FD38BDC0466B
:10018000873A0000B80400108D3A0000943A00004D
:100190009A3A000008B5074B0120196801F0E4FA0B
:1001A000012001F0C1FA02F04DFE012001F0CCFA6D
:1001B00008BDC046B004001010B5041C0D2107484E
:1001C0000C2200F09BFC00F0FBFB201C0021032212
:1001D00000F00AFD00F0FEFB10BDC0461F3C000011
:1001E00013B59620000201F035FB1248FFF7E4FF3B
:1001F000FFF7D0FF1048114901F010FD002401F075
:10020000CFFB002802D001F005F800240A2001F0FD
:100210002BFA684601A9FFF753FF009B002B03D17F
:10022000074B01349C42EADDFFF7B4FF054801F0BB
:10023000F5FC13BDA63A0000B53A0000C03A000034
:100240006F170000C73A000000B5074B89B01A7855
:10025000064B68461B78064901F0EBFC6846FFF741
:10026000ABFF09B000BDC046B8010010000000108F
:10027000D23A000013B5FFF7E7FFFFF78BFF00242A
:10028000684601A9FFF71CFF009B002B2CD0182B00
:1002900021D004DC142B0DD0152B20D104E0342BFD
:1002A00012D0352B1BD107E0134B00241A783E2ABD
:1002B00016D806E0104B08E0104B00241A78062AE6
:1002C0000ED801321A700BE00C4B1C78002C07D0B2
:1002D000013C1C7003E0FFF75DFF282400E00024D0
:1002E00000F05AFBFFF7B0FFC820013401F0BCF961
:1002F0001D2CC5DD13BDC046B80100100000001064
:1003000073B5124B041C1249186803F025FB114900
:100310000090114A114B201C01F08BFC00F0C4FD31
:10032000002812D000F0DCFDFA218900051C03F042
:1003300013FB061C201C01F0C9FC094B2018734359
:100340000849EB18321C01F074FC73BDB4040010B2
:1003500040420F00E03A0000C03A0000ED3A0000D1
:1003600018FCFFFFF03A000070B50D1C161C041CB1
:1003700000F026FB0B480D210C2200F0BFFB281CCF
:10038000A1B2002200F030FC07480321062200F051
:10039000B5FB301C0121092200F026FC00F01AFBFD
:1003A00070BDC0461F3C00005C3B000010B588B02B
:1003B000041C6846FFF7A4FF69466A46201CFFF745
:1003C000D3FF08B010BD000073B518200021FFF75F
:1003D00085FE424E0024424D983600E0404D0120FB
:1003E00001F0B2F9002C01D0002000E0062001212C
:1003F00001F00AF9684601A9FFF762FE009B002B95
:1004000021D1002CF0D13368002B0DD0354B009456
:100410001A6811321A6004E002F0BEFC009B01333E
:100420000093009B102BF7DD2F4BED18DED5182025
:100430000021FFF753FE294B94331C6863425C4153
:1004400000F072FACEE7002C03D0182BC7D100F0D1
:10045000C9FA009B182B2BD1019B00220192822B01
:1004600022D004DC322B0ED0732B20D119E0832B49
:100470000FD0C22B1BD11D4B196801311960022905
:1004800016D11A6014E01A4B01201B68C01A00F044
:1004900039FD0120FFF78AFFFFF77CFEFFF717FE0B
:1004A00006E0FFF79DFE03E0FFF7E4FE00E00193A6
:1004B000104B0120196801F057F9012001F034F9BF
:1004C0000098019902F026FD044B002494331B6828
:1004D000002B83D100F028FA01247FE7B804001034
:1004E00020BF0200E40200100CFEFFFF900100108C
:1004F00008000010B004001013B501F017FC00F064
:10050000BDFB00F06FFA1C48002100F01DFF002128
:100510001A4800F019FF00F057FC002004210122C6
:1005200000F0A0FE0020021C042100F0E9FE0020E3
:100530000521012200F096FE00200521021C00F09A
:10054000DFFE00F073FE3C24201CFFF72FFF013C70
:100550001E2001F089F8022CF6D102F03FFB1E2389
:10056000009310230193064806490022064B02F02F
:10057000EFFBFFF729FFC046984004409C40044031
:1005800009380000C1000000E402001000B500E0DE
:1005900001300378202BFBD000BD00B5031C303B9D
:1005A000DAB2092A01D8181C08E020231843031CDA
:1005B000613B5738052B01D90120404200BD70B581
:1005C0000E1CFFF7E3FF0025041C06E0FFF7E5FF24
:1005D000002805DB2D010543013420780028F5D1E2
:1005E0003560201C70BD000008B500F079FC011CCE
:1005F000014801F013FB08BDFB3A000000B5C30041
:10060000181A064BC0180723013BC25C002A03D10D
:10061000002BF9D1012000E0002000BD540500109E
:100620007FB5194801F0FAFA00250326354219D1A1
:10063000281CFFF7E3FF002810D0681CFFF7DEFF3F
:1006400000280BD0A81CFFF7D9FF002806D0E81C13
:10065000FFF7D4FF002801D004350FE00B48291C18
:1006600001F0DCFA291C684601F0CAFB6846FFF776
:100670004BFD074801F0D2FA6C1C251CFF2DD5DD7F
:10068000FFF750FD7FBDC046C03A0000073B0000A9
:10069000D35F000070B50E1CFFF778FF0D25041C1A
:1006A0002078FFF77AFF002807DB01347055013D01
:1006B000F6D2201CFFF76AFF00E0002070BD0000AA
:1006C00030B5464C87B023680868002B06D14448F3
:1006D00001F0A4FA02F082FA012357E0012B12D1B3
:1006E0008379202B07D0002B05D03E49062201F04C
:1006F00000FB002803D1394B1A6801326AE03A48FE
:1007000001F08CFA5EE00378412B1BD1374C0230AC
:10071000211CFFF7BFFF002854D00378422B51D192
:10072000211C02300E31FFF7B5FF00284AD00378B4
:10073000432B47D1211C02301C31FFF7ABFF0028AF
:1007400049D13FE04D2B23D1294D0230291CFFF721
:10075000A1FF002836D003784E2B33D1291C02305C
:100760000E31FFF797FF00282CD00378472B29D1B3
:10077000023005A9FFF723FF059B002B22DB2A3D52
:100780006B651C481C4901F049FA0023236022E0F4
:1007900005A9FFF714FF0378041C202B01D0002BC0
:1007A00010D10025201C01A9FFF774FF0599041C36
:1007B000691801A801F038FB002C03D00135042D85
:1007C000F0D108E002F00AFA0A480C4901F026FAD2
:1007D000024B00221A6007B030BDC046BC020010B8
:1007E000103B0000C03A0000263B0000B804001097
:1007F000E2040010323B00003C3B00003F3B0000A5
:1008000037B54C6824E0201CFFF7C0FE01A9FFF7B4
:10081000D6FE019B041C002B1DD0D8B2FF2B09DD96
:1008200000F0FCF9051C01980012C0B200F0F6F9C6
:10083000019003E000F0F2F90025019001980028F2
:1008400002D0291CFFF74AFC23785A1E9341E41872
:100850002378002BD7D137BD08B5064A012113787C
:100860004B40137001D0044900E00449044801F0F2
:10087000D5F908BD9D030010463B0000493B000030
:100880004D3B000070B5051C01200821021C00F042
:1008900037FD0724012601200821002200F030FD49
:1008A0002A1C224132400020022100F029FD0120B3
:1008B0000821021C00F024FD013CECD270BD10B5F3
:1008C0000021041C0A1C022000F01AFD201CFFF766
:1008D000D9FF10BDF7B5012300930023019372B631
:1008E0006C46061C02AF01CC50235B421843C0B2D9
:1008F000FFF7E5FF0020FFF7E2FF1020FFF7DFFF23
:10090000E020FFF7DCFF002502200021012200F09B
:10091000F7FC705D0135FFF7B5FF842DF4D1843607
:10092000BC42E0D162B6F7BD08B5AC20FFF7C7FF07
:10093000AE20FFF7C4FFA520FFF7C1FF08BD38B503
:100940000D1C041C012200F08DFC291C201C01221E
:1009500000F0D6FC38BD08B5AF20FFF7B0FFA420EB
:10096000FFF7ADFF08BD08B5AE20FFF7A8FF08BD33
:1009700010B5041CF820FFF7A2FF201CFFF79FFF13
:1009800010BD10B5041C8120FFF799FF3F202040C7
:10099000FFF795FF10BD000008B5074B20201B781E
:1009A0001843FFF78CFF0A2000F05EFE034B187817
:1009B000FFF7E7FF08BDC04600000010B8010010B7
:1009C00008B5842202480021520001F05FF908BDF9
:1009D000A503001008B50248FFF77CFF08BDC0461C
:1009E000A503001008B501200821FFF7A8FF00208B
:1009F0000221FFF7A4FF02200021FFF7A0FF022041
:100A00000621FFF79CFF0320011CFFF798FF03203E
:100A1000011C002200F074FC02200621002200F0DC
:100A20006FFC06210122022000F06AFCFFF7C8FFDC
:100A3000FFF7D0FFA220FFF742FFA020FFF73FFF04
:100A4000C020FFF73CFF0020FFF792FF0A2000F0D4
:100A50000BFE4020FFF733FF2C20FFF730FF322042
:100A600000F002FE2E20FFF72AFF322000F0FCFDEE
:100A70002F20FFF724FF0A2000F0F6FDFFF78CFF80
:100A8000AF20FFF71CFFA420FFF719FF08BD0000EF
:100A900000B50F290ED883280CD8CB0884225343E5
:100AA0000722C0181140044B80220A41111C1A5C15
:100AB0001143195400BDC046A5030010F0B55B18E2
:100AC000DBB216E08425CC086C4307270F40802555
:100AD00004193D41EFB2A6189C4605E0064BE51807
:100AE0002B7801343B432B70B442F7DB0131634672
:100AF000C9B29942E6D3F0BDA503001000B5074B7B
:100B00001860074B1970074BD1081A70064B197003
:100B1000500701D00131197000BDC046A00300107C
:100B2000AD040010AE040010A4030010F0B589B0AD
:100B3000059106925A2800D92020284B284A1B6884
:100B400093420BD1440003212418623C019103918C
:100B50000EE0195D01320231641802E00024221C0B
:100B600020388242F5D31A5D1B195B7801920393FA
:100B700000252CE06B430199FA188A4215D2174AD6
:100B800000261268D2191219D3189B7804930123F6
:100B9000049AB340134205D0029B07989919C9B231
:100BA000FFF776FF0136082EF1D1029B013708339B
:100BB000DBB2029306E0059A06995319DBB2029163
:100BC0000027079307490B789F42D3D30135039A37
:100BD0009542F0D109B0A8B2F0BDC046A003001004
:100BE0005C3B0000A4030010F7B5061C0C1C01922E
:100BF00001F06CF800250090832708E06B46705DDB
:100C0000E1B21A79FFF792FF013024180135A742AB
:100C100002D3009B9D42F1D3F7BD000000B50F2326
:100C2000020918408000031F00D52833002B0EDB7B
:100C3000511E0320884280414042002807D1242BC6
:100C400006DC04218A1A0349CB18985C00E00020D6
:100C500000BDC0462240000070B5064E051C0024B1
:100C6000A05D054B291CC018013400F06DFB0A2C57
:100C7000F6D170BD5E40000000400440F8B5102081
:100C8000FFF7EAFF094C271C143725786678281CE3
:100C9000311C002200F0E6FA0234281C311C01222B
:100CA00000F02EFBBC42F0D1F8BDC0464A40000027
:100CB000F8B50B4C271C143725786678281C311C96
:100CC000012200F0CFFA0234281C311C002200F06F
:100CD00017FBBC42F0D10020FFF7BEFFF8BDC046B5
:100CE0004A400000F0B589B0002404900591FFF758
:100CF000C5FF0220072101220694079400F0B2FAF2
:100D000002200721221C00F0FBFA201C0B2100F01E
:100D1000CDFAA04202D11823069301240021264DCA
:100D200003916A782F78111C0192381C012200F07F
:100D300099FA381C0199002200F0E2FA03231F4EB1
:100D4000029314E03078717800F0B0FA002807D1EF
:100D500003991B4AA3008A5C183369465A50013430
:100D6000029A039B013A013302920393023EE30F7E
:100D700000210122A2424B41DBB28B4202D0029BF6
:100D80008B42DFDA381C0199002200F06BFA0199DE
:100D9000381C012200F0B4FA0A4902358D42C0D154
:100DA000201E06D0069B049A05991360079B01201C
:100DB0000B6009B0F0BDC0464A4000002040000072
:100DC000224000005E40000008B50120021C0B21FB
:100DD00000F048FA01200B21002200F091FA0320D4
:100DE0000221012200F03EFA03200221002200F03D
:100DF00087FA08BD37B5234B10211A68051C8A43B2
:100E00001A60214B8022196892010A431A6001205E
:100E10000B21002200F026FA01200B21002200F015
:100E20006FFA1A4B9F211A68194C8A431A601A6884
:100E300018491A60184B186802F08EFD80230002D2
:100E400018432A1C20600221032000F059FA1420C4
:100E500000F00AFC2368FF229343236023680F4AB3
:100E6000134323600E4B1A680192019A002AFADAA2
:100E700022680C4B13402360FFF7A6FF0198000483
:100E8000800D3EBD3882044080800440984004407C
:100E900000C0014000093D00B404001080000001C2
:100EA0002CC00140FFFFFFF810B50C4C2068002853
:100EB00013DA00202060FFF79DFF0A280ADC0120DA
:100EC000FFF798FF0138C023FF385B00984201D834
:100ED00001232360FFF778FF206810BD0400001095
:100EE00008B5FFF7E1FF011E08D00120FFF782FFE0
:100EF000011E03D0024802F02FFD011C081C08BD92
:100F000050BB120010B500280DD0254B80211A6867
:100F10008A431A60234A012311681942FCD0224BEC
:100F200003221A6001E0204B1860204B01220021AF
:100F30001A6019601A6019681142FCD01C4B01221A
:100F40001A601C4A802114684902214311601A1C4E
:100F5000002804D1124B8024196821431960164BD4
:100F6000196888421AD01860002801D0134800E0A0
:100F70001348116802F0A2FC124C2121206002F0FB
:100F8000EBFC114B18609620000200F063FCFA2184
:100F90002068890002F0E0FC00F04CFB10BDC04668
:100FA000388204400C800440708004407480044007
:100FB000788004408080044008000010006CDC024F
:100FC000001BB700B4040010B004001008B500F016
:100FD0003BF9134B00211A68120B12031A60114BD4
:100FE0001A68120B12031A600F4B1A68120B1203C5
:100FF0001A600E4B1A68120B12031A600C4B012276
:1010000019600C4B1A6019601A6019681142FCD003
:10101000094B23221A600120FFF774FF08BDC04668
:10102000008000500080015000800250008003507A
:1010300040800440448004400880044070B50F495B
:101040000F4800F0EBFD0F4800F0E8FD0E4E0F4D8D
:1010500000242B196159DA68301C0A4B143400F053
:10106000DDFD782CF5D10A4800F0D8FD00F018FB22
:10107000011C084800F0D2FD70BDC046C03A000017
:1010800068400000B9400000794000000C000010EA
:1010900084400000A6400000F0B53C4B8BB01D68BA
:1010A000002D3AD03A4B02901B6801209B685DE00E
:1010B00001342378202BFBD0002B3AD0B300083327
:1010C0006A469C500136FF2D01D135E0013423786A
:1010D000202B01D0002BF9D1202B02D1002323702B
:1010E0000134012E1BD12A4F2A4B07223B6001926B
:1010F0003D1C09E02B680298196800F009FE0028E1
:1011000008D02B6814332B60019B013B0193002B0B
:10111000F0D132E03B681D7901E0041C2E1C2378DD
:10112000002B06D000230722B2425B41DBB2002B2A
:10113000BFD1002E1CD000E00025154C022E05D199
:101140000398154900F0E4FD002801D0AE420AD80A
:1011500023681248D96800F061FD236810481969B6
:1011600000F05CFD04E02368F0B29B6802A9984798
:10117000064B1B68002B07D103E00198011CFFF709
:101180005DFF084800F04AFD0BB0F0BDBC02001046
:10119000C40200100C000010B3400000B540000075
:1011A000373B0000BC40000038B5041C154D0A2830
:1011B00008D002D808281CD110E00D2802D07F28C2
:1011C00017D10BE02B6800221A700F4800F026FDA3
:1011D0000E4C201CFFF760FF2C6012E02A680B4BBE
:1011E0009A420ED90A48211C00F018FD2B68013BD9
:1011F00006E00748211C00F011FD2B681C7001332C
:101200002B6038BDC0020010B9400000B9010010C9
:10121000C840000008B503E000F0A0FBFFF7C4FFE2
:1012200000F0BEFB0028F7D108BD000008B5034A56
:10123000034B04481A6000F0F1FC08BDB90100102E
:10124000C0020010BC400000044B40211A680A4351
:101250001A60034B01221A707047C0468080044018
:10126000C802001070B50E4B061C1B780D1C141C18
:10127000002B01D1FFF7E8FF013E022E03D8094BF6
:10128000B600F35800E0084B1A68012C03D1AC40BB
:1012900014431C6003E00124AC40A2431A6070BDFB
:1012A000C80200104C4100000080005038B50F4BC0
:1012B000051C1B780C1C002B01D1FFF7C5FF00207B
:1012C000032D11D8281C012302F0E4FA02040608B9
:1012D000074A04E0074A02E0074A00E0074A1068AC
:1012E000A3401840431E984138BDC046C8020010B4
:1012F000FC3F0050FC3F0150FC3F0250FC3F0350BC
:1013000070B50E4B061C1B780D1C141C002B01D154
:10131000FFF79AFF013E022E03D8094BB600F3589F
:1013200000E0084B1A68012C03D1AC4014431C6048
:1013300003E00124AC40A2431A6070BDC802001053
:1013400058410000FC3F005038B5084B041C1B7886
:101350000D1C002B01D1FFF777FF23681822934360
:10136000236023681D43256038BDC046C8020010B5
:101370001F234209184001238340181C014B92008F
:10138000D050704700E100E01F23420918400123BC
:101390008340181C2032024B9200D0507047C04648
:1013A00000E100E0054B3F221A60054B01221A6064
:1013B000044B40211A688A431A6070472480044015
:1013C000D88004403882044008B5044B40211A6894
:1013D0008A431A60FFF7E6FF08BDC0463882044022
:1013E00008B5154B1868FFF78DFD0720FFF7CCFFF8
:1013F0000820FFF7C9FF0A20FFF7C6FF0C20FFF700
:10140000C3FF0B20FFF7C0FF0920FFF7BDFF0B4A0A
:101410000023136001210A4A49421160094A1360FE
:10142000094A1360094B01221A60094B1A680132FC
:101430001A60C04608BDC04608000010048204407F
:101440000882044004C000403CC0004000C000408E
:10145000CC02001008B5FFF72BFC0A480021FFF76B
:1014600073FF09480021FFF76FFF08480021FFF7CD
:101470006BFF07480021FFF767FF06480021FFF7D1
:1014800063FF08BD0840044000400440AC400440F5
:10149000144004401C400440F8B5071C0C1C72B6F4
:1014A000FFF7D8FF434B1A68434B1A60002F01D057
:1014B000424B00E0424B434A04211360424B434DF0
:1014C0001A680A431A6000232B609C4218D0072038
:1014D000FFF74EFF0820FFF74BFF0A20FFF748FFFA
:1014E0000C20FFF745FF0B20FFF742FF384B394A2E
:1014F00019680A401A602A68EC235B0113432B60C9
:10150000002F4FD0344B354C354900260E60201C3F
:101510001E60311CFFF718FF301C0921321CFFF739
:10152000A1FE301C0921321CFFF7EAFE2D4B802260
:10153000196811431960236807218B4323602368CE
:1015400002210B4323607B00DB1999015B189B0090
:101550002549DF19254B0F6003211960244B2549CC
:10156000186801401960196809200A431A60FFF7DA
:10157000FFFE174A802311689B00194311602A68F7
:10158000022113431C4A2B60012313601B4A116084
:101590001B4A134913601660136010681842FCD090
:1015A00001230B60174B012252421A6062B630BF12
:1015B000F8BDC0463882044034820440BF180000A1
:1015C000FF1800003082044010ED00E00482044067
:1015D000008204407FE2FFFF044001406440044079
:1015E00004C000408080044018C0004014C0004087
:1015F0003CC000400FF0FFFF788004407080044042
:10160000748004400882044008B5FFF745FF08BD18
:1016100000B5064B1A6801321A601B68013303D10A
:10162000034B1A6801321A6000BDC046D402001094
:10163000D002001000B5074B98420AD8064A002392
:101640001360064A01381060054A1360054B0722F3
:101650001A6000BDFFFFFF00D402001014E000E09C
:1016600018E000E010E000E000B50C4A1368002824
:1016700000D10120C1438B4204D809E011688142A6
:10168000FCD301E0591C081811689942F6D203E016
:101690001168C91A8142FBD300BDC046D4020010B4
:1016A00010B5064BFA211868054B89001C6802F03A
:1016B00005F9044B5C43201810BDC046D40200104D
:1016C000D002001037894100034B01221A60034BFE
:1016D0001A6801321A60704700C00040D80200103A
:1016E000034B01221A60034B1A6801321A607047DB
:1016F00000000140DC020010034B01221A60034B82
:101700001A6801321A60704700400140E002001080
:10171000034B01221A60034B1A6801321A607047AA
:1017200000800140E402001000B5002803D1044B02
:1017300001221A6003E0012801D1024B186000BDAC
:10174000044001400480014000B5002802D1044B50
:10175000186004E0012802D1024B00221A6000BD8B
:10176000044001400480014010B500280FD1124B05
:1017700080221C68920022431A60104B03221860DA
:101780000F4B19600F4B1A608022D20211E0012822
:1017900011D1094B80221868D20002431A600A4B0B
:1017A00000221A60094B03221960094B1A6080223B
:1017B0001203084B1A6010BD80800440E002001044
:1017C0001840014014400140E4020010188001401C
:1017D0001480014000E100E008B5184B1A680E23A0
:1017E0001340062B0DD1164B9E221B68DBB2134211
:1017F00004D0144A5360144B1B681EE0D9071CD553
:1018000001E0042B05D1104B1868C0B200F0B7F806
:1018100013E00C2B06D10B4B8022596852000A436F
:101820005A600AE0022B08D1054B1A68054B910655
:1018300001D5002200E001229A6008BD0880004026
:1018400014800040E802001000800040004870470B
:10185000E802001070B52A4C2A4B80229203DA6706
:1018600000219022061C201C00F010FA0023A36027
:1018700000F06EF8244B07251A68244CAA431A601E
:101880001968012211431960214B1968A943196095
:101890001968114319601F4B8021186849010143E1
:1018A00019601D4B1A608322226019681B4B18684F
:1018B00002F004F8311C000902F000F81849030A8C
:1018C000184A0B60C0B2032310602360164B1D60E2
:1018D000164B186860201C680440602CFBD101E0A6
:1018E000146800E001201C680442F9D1044B012275
:1018F0001A700F4B802292031A6005230B6070BD93
:10190000E802001004E100E0A44004400C80004024
:10191000A84004408080044098800440B404001033
:101920000480004000800040088000401480004097
:1019300000E100E000B5044A202311681942FCD000
:10194000024B186000BDC04614800040008000407B
:1019500008B5FFF77BFF0023437308BD08B5FFF709
:1019600075FFC27B031C8218107CDA7B7F21013259
:101970000A40DA735A7B013AD2B25A7308BD10B5E5
:10198000041CFFF763FF837B7F22C3181C74837BD7
:10199000013313408373437B0133DBB2437310BDC8
:1019A00008B5FFF753FF407B431E984108BD30B593
:1019B000002402E00570013401301D5D002DF9D1D5
:1019C000121B131C02E00170013B0130002BFADCFA
:1019D000D043C0170240A01830BDF8B5051C0F1C3D
:1019E0001E1C541E092B01D800240FE0181C0A21CC
:1019F00001F064FF221C031C391C281CFFF7EDFFBB
:101A0000041C2D1805E02F7001340135013A002A1D
:101A1000F9DC301C0A2101F095FF30312970601C7F
:101A2000F8BDF8B50C1CD9175F18061C4F40551EA1
:101A3000092F12D9381C0A21002B03DA01F03EFFCE
:101A4000434202E001F03AFF031C211C2A1C301C17
:101A5000FFF7E7FF041C351813E0002B00DA951E92
:101A6000002201E0B4540132A91A0029FADCEC4347
:101A7000E4172C403519002B03DA2D232B70013489
:101A80000135381C0A2101F05DFF30312970601CDE
:101A9000F8BD73B5069E041C1D1C3009531E00289A
:101AA0000AD000901A1C201C2B1CFFF7F2FF2418F0
:101AB00005E0217001300134013A002AF9DC0F23DE
:101AC0001E40092E01D8303604E0002D01D03736F3
:101AD00000E057362670013076BDF0B585B0041CA5
:101AE0000F1C002801D00021017000256BE0252982
:101AF00003D021700132013405E05178252904D149
:101B000021700232013401355DE0302903D0013209
:101B10000292202101E002320292029E9C4632781B
:101B20002D3A50424241B6180296002205E00A239F
:101B30005A438218303AD2B201363078031C303B17
:101B4000092BF4D90296AE186346BE4201D97A1B1E
:101B5000D2B269280ED006D863282CD0642809D0C8
:101B600058283ED119E075280AD078280FD073285C
:101B700037D11AE01E1D201C1B68FFF752FF04E03E
:101B80001E1D201C1B68FFF728FF331C17E01E1DBD
:101B90001B68201C0093002304E01E1D1B68201CF2
:101BA00000930123FFF775FFEFE71E1D201C1B6844
:101BB000FFF7FDFEE9E71A68012022700433029A5C
:101BC000241801322D181178BD4201D200298ED17E
:101BD0000023BD4201D2237005E0013C2370013D8A
:101BE00001E001256D4205B0281CF0BD10B50C1CAC
:101BF000131C6421221CFFF770FF10BD00B5031CED
:101C00009BB00A1C01A8191CFFF7F0FF632800DD38
:101C1000FEE701A800F0A6F81BB000BD0FB407B5A1
:101C200004A901C90191FFF7E9FF03B008BC04B0A2
:101C300018470EB403B503AA02CA0192FFF7D6FFF4
:101C400002B008BC03B0184770B50323041C184247
:101C500005D10D1C041C194201D1934201D300236C
:101C600011E0131C40CD043B40C4032BFAD8141FD1
:101C7000A4080134A400032309191A400419EEE74B
:101C8000CD5CE55401339342FAD170BD30B50B04FD
:101C90000D061D430D430B021D430323041C9342F9
:101CA0000DD218420BD1131C043B20C4032BFBD8CC
:101CB000141FA4080134A40003231A4004190023AC
:101CC00001E0E15401339342FBD130BD00B5002364
:101CD00000E00133C25C002AFBD1181C00BD00B536
:101CE000031C01E0013101330A781A70002AF9D18E
:101CF00000BD30B5031C002406E01D5D085D281AF8
:101D000005D10134002D02D09442F6D1002030BD1F
:101D100000B502E00130002B06D00A7803780131CB
:101D20009342F7D0981A00E0181C00BD08B5FFF7E1
:101D30004DF90B4BFA211868890001F00DFEFFF7F1
:101D400079FCFFF781FAFFF73FFB96200002FFF7CF
:101D500081FDFEF747FEFEF733FEFFF767FA08BD89
:101D6000B404001010B5041C02E00134FFF7E2FDDA
:101D700020780028F9D110BD30B5F8238A01DB00A6
:101D800013404A05920E1343F822120211401943E0
:101D90000A235943CA1083181C1CEB345D7824783D
:101DA000EA336C401B7824021C43835C201C58409F
:101DB0000723194008418005800D30BD08B5054B4B
:101DC000011C984201DD044BC1180448EA38FFF7B2
:101DD000D3FF08BDFF17000000F8FFFF64410000BB
:101DE00008B54018511A013101F018FE08BD08B5B8
:101DF000801889189A1A0132FFF726FF08BD0000E3
:101E000010B5CB00591A074B0F22C9180023CC5C20
:101E100014400470CC5C0133240944700230072B59
:101E2000F5D110BD5405001010B5CB00591A064B62
:101E3000C91800234278047812012243CA5401339E
:101E40000230072BF6D110BD5405001030B5B14B50
:101E500087B0D96EB04D4A1E91416A46D175A96AC4
:101E60001A1CC806400F0138062807D801F012FDD9
:101E7000040C1F1217191C00022409E05A6E1632B6
:101E80009200D3581C1C15E05B6E16339B00D4588F
:101E900000230FE09B6DD46DA3420ADC0AE002240C
:101EA00003E00C24032305E00D24231C02E00D2491
:101EB000EEE70D242C6148111F2800D922E16A4663
:101EC0001732944901F0F0FC2000220028002A007B
:101ED0002D002F00380040004400490051005F00F1
:101EE00067006F00770085009300A200B400C30074
:101EF000D500D300E300E600E900F100010105018F
:101F00000F01110113011901081C00E08348191C7D
:101F1000221CFFF765FFF5E08148F8E70A1C0E3246
:101F200003E07E4809E00A1C1C32081C111C1A1C24
:101F3000231C01F0F9F8E5E07948011C0E391A1C60
:101F4000231CFFF754FFDDE07448011C0E31EEE75F
:101F50000A1C1C32081C111CF1E70A6E1020002A12
:101F600000D00A200A1C0E3206E00A6E1020002A59
:101F700000D00A200A1C1C3200946C4617340290D0
:101F80000194081C51E001201070086E10220028F6
:101F900044D00A2242E00A6E1020002A00D00A2013
:101FA0000A1C0E320EE001201070086E102200286C
:101FB00055D00A2253E00A6E1020002A00D00A20D1
:101FC0000A1C1C3200946C46173402900194081CC1
:101FD00078E00A6E1021002A00D00A21504A684693
:101FE0001730019002910094101C111C1DE00A6E24
:101FF0001020002A00D00A20494A00946C46111C87
:10200000173402901C390194101C0EE0096E012057
:1020100010701022002900D00A224149684617306A
:10202000019002920094081C002201F087F869E0F8
:102030000A6E1020002A00D00A20394A00946C460B
:10204000111C173402901C390194101C3AE0096EDF
:10205000012010701022002900D00A223049684661
:102060001730019002920094081C00222AE00120FF
:1020700010700A6E1021002A00D00A21284A6846F2
:102080001730019002910094101C00211AE0009278
:1020900022481CE00092224819E00A6E1020002A13
:1020A00000D00A200A1C1C3206E00A6E1020002A0A
:1020B00000D00A200A1C0E3200946C46173402909D
:1020C0000194002001F063F81CE00092081C00213C
:1020D00004E00D1C1C35081C0092291C1A1C231C32
:1020E00001F0B0F80EE0081C02E00C4800E00C48DB
:1020F000191C221C01F0BFF804E0081C221C191C4A
:1021000001F0C4F86B46DA7D024B07B00120DA66B5
:1021100030BDC046B8040010540C0010C6040010B6
:10212000D404001010B506490B1C88331A68141C1F
:102130001E34A4006050013203210A401A6010BD11
:10214000B8040010054B0320191C88310A68013AB5
:1021500002400A601E329200D0587047B804001046
:10216000F8B5114D2C1C8C3420680130FFF726FE89
:102170000E4B0122D8629F6AAB6E061C02409A4247
:1021800010D1830703D420680230FFF7CBFFFF2371
:102190009B001E40B601BF10044B8C353743012213
:1021A0002F60DA600220F8BDB8040010540C001053
:1021B00030B50C4B0C489A6A031C8C331C68D30551
:1021C0009B0E910500D5403B856E921001210A407F
:1021D000AA4204D1E3188C300360024BD96001207D
:1021E00030BDC046540C0010B804001008B5084BB0
:1021F0005A1CD07F9A1CD27F000112021043DA7F52
:102200000333DB7F10431B031843FFF78BFF08BD2D
:10221000B804001038B5FFF795FF064903230F22D5
:10222000051C5C181540013325770011072BF7D1E9
:1022300038BDC046B804001008B5FFF783FF034B54
:1022400001228C331860024BDA6008BDB80400101C
:10225000540C001010B5064CA36E002B06D0FFF7EF
:1022600071FF044B8C3401222060DA6010BDC0463F
:10227000B8040010540C001010B5064CA36E002BCF
:1022800006D1FFF75FFF044B8C3401222060DA6037
:1022900010BDC046B8040010540C001008B5124B15
:1022A0001B68002B00D09847104B5A69002A15DD97
:1022B000012A07D1DA69002A04D09A610022DA6182
:1022C0000A225A615B690322191C91430A1E02D03B
:1022D000074A0121D166054A013B5361044B903303
:1022E0001A68024B5A6208BD78030010540C0010A3
:1022F000B804001000B5064B5A69002A07DD9A6938
:102300000F21044B1140D97712110133DA7700BD48
:10231000540C0010B8040010044B597F9A7F090137
:1023200012020A43197F0A435A677047B804001023
:1023300030B50B1C093B012B0FD8084A00239C1811
:10234000257FC45CA54205D0054B08395A68114366
:10235000596002E001330E2BF1D130BDB8040010FA
:10236000540C001008B50E4B1B68292B17D00829F8
:102370000DD0192913D1427808231A4202D0002225
:10238000027002E00F2303700723437005E000236F
:102390001A1CC25401330E2BFBD1FFF745FD08BDBB
:1023A000540C00101FB50D4B5C6F002802D00F229B
:1023B000944304435C676846211CFFF721FD68468F
:1023C000211CFFF7CFFF054A00236C46185D9918C2
:1023D000013308770E2BF8D11FBDC046B80400109A
:1023E0001FB5124B0F225C6F944304435C67104B84
:1023F0001B68292B01D0082C17D06846211CFFF739
:10240000FFFC6846211CFFF793FF084A0023991838
:10241000097F6846195401330E2BF8D1211CFFF7B0
:10242000A1FF6846211CFFF7FFFC1FBDB804001088
:10243000540C00101FB5114B114C1B68292B02D0F6
:10244000636F082B18D0616F6846FFF7D9FC616F86
:102450006846FFF76DFF0A4C00231A19127F694680
:102460005A5401330E2BF8D1616F6846FFF77AFF9B
:10247000616F6846FFF7D8FC1FBDC046540C0010C2
:10248000B804001010B50D4C631CD87FA31CDB7F73
:1024900000011B021843E37F1843E31CDB7F1B038F
:1024A0001843FFF78BFC0F23021C1A4022770211FE
:1024B000134000126377A07710BDC046B804001027
:1024C000044B5A6E16329200D258121A51424A41A7
:1024D000DA667047B804001000B5064B5A6E163223
:1024E0009200D1580139D150002901DA0D21D15083
:1024F00000BDC046B804001000B5064B5A6E163237
:102500009200D1580131D1500E2901D10021D15072
:1025100000BDC046B804001000B5094B5A6E163213
:102520009200D2580D2A03D11A1C2932127805E0E4
:102530009A18507F117F0001021C0A435A6500BDA2
:10254000B804001010B5084B0F245A6E16329200D2
:10255000D1585A6D58181440013104770D2902DC06
:102560005B1812111A7710BDB804001030B50F4B6C
:102570005A6E596D16329200D2580D2A07D11C1C82
:1025800029342478F02008402043586507E0981843
:10259000447F057F24012C435C650B114377034B7B
:1025A0009A180F231940117730BDC046B8040010A7
:1025B00008B504480022011C1C390D23FFF717FC45
:1025C00008BDC046F004001008B504480022011CF4
:1025D0001C310D23FFF70BFC08BDC046D4040010CE
:1025E00008B504480022011C1C310D2300F09CFD9D
:1025F00008BDC046D404001008B504480022011CE0
:102600000E390D23FFF7F3FB08BDC046E2040010AE
:1026100008B504480022011C0E310D23FFF7E7FB2B
:1026200008BDC046D404001008B504480022011CAF
:102630000E310D2300F078FD08BDC046D404001013
:102640000C4A0023111C46310B70111C47310B70D2
:10265000111C48310B70111C49310B70111C4A318F
:102660000B70111C4B310B70111C4C314D320B7027
:1026700013707047B804001000B5074A011C04230A
:1026800000208A1804E0D118463109784000084338
:10269000013BF8D200BDC046B804001030B5074A6F
:1026A00000238918012206E0CC18051C4634154089
:1026B000257040100133042BF6D130BDB804001052
:1026C00038B50020FFF7D8FF084C051C0021207FFB
:1026D000FFF7E4FF25770420FFF7CEFF0421051C58
:1026E000607FFFF7DBFF657738BDC046B804001098
:1026F00010B50020FFF7C0FF034C20770420FFF740
:10270000BBFF607710BDC046B804001010B5054C83
:102710000021207FFFF7C2FF607F0421FFF7BEFF8B
:1027200010BDC046B804001010B5094C231C8C33F2
:1027300018680130FFF742FB064B021CD8620F23DA
:102740001A4022770211134000126377A07710BD60
:10275000B8040010540C001010B5094C0021201CC6
:102760000D22FFF73DFB201C0E3000210D22FFF74C
:1027700037FB201C1C3000210D22FFF731FB10BD60
:10278000B804001010B50C4B00211A1C187F1C78DF
:1027900001312043187701330E29F7D1936E002BB6
:1027A00008D0064B1B690D2B04D1137F111C293156
:1027B0000B70537310BDC046B8040010540C0010C9
:1027C00010B50C4B00211A1C1C7F187801312040D9
:1027D000187701330E29F7D1936E002B08D0064BE2
:1027E0001B690D2B04D1137F111C29310B705373FE
:1027F00010BDC046B8040010540C00107FB5002373
:102800000C4A0D251C1C1118097F01306E46995584
:10281000C60F8542664176420133111C30400E2BB3
:10282000F1D100236C46185DCA18013310770E2BC6
:10283000F8D17FBDB804001010B5074B5A6E1632A0
:102840009200D1585C1801392077D150002901DA63
:102850000D21D15010BDC046B8040010034A00231A
:10286000111C943198320B6013607047B80400104B
:10287000034B012194331A684A401A607047C046DE
:10288000B8040010044A002313678C321360034B12
:102890000122DA607047C046B8040010540C0010E2
:1028A00008B59A4B0F20996A994A8B1018408911E4
:1028B000013852560E2800D9C1E000F0EBFF081194
:1028C0001A2327C02EC0C037C0C0C03B3F00002A1B
:1028D00000DAB4E08F4B9A18403200239371A9E0DC
:1028E000002A00DAABE08B4B01209A18403290713D
:1028F000A4E0002A00DAA2E0864B9A1840329279CE
:10290000DA6697E0081CFFF797FF93E0002A00DAE9
:1029100095E0101CFFF7D4FD8CE0002A00DA8EE071
:102920007C4B596E16318900CA5083E0081CFFF7B2
:1029300057FD7FE0081CFFF735FD7BE0002A00DA39
:102940007DE0101CFFF75AFF74E0724B01209833B2
:10295000186073E0FFF7E0FD6CE0FFF793FF69E0BC
:10296000FFF726FE66E0FFF7EDFD63E0694B00220E
:102970005A665FE0FFF728FE5CE0FFF7F7FD59E0DD
:10298000644B0120586659E0FFF72AFE52E0FFF73A
:10299000CBFE022052E0FFF72FFE4BE0FFF726FCB4
:1029A00048E0FFF735FE45E0FFF7D6FE42E0FFF7CF
:1029B00031FC3FE0FFF738FE3CE0FFF79BFC39E0DD
:1029C000544B00221A6635E0FFF7A6FC32E0514B6B
:1029D0000120186632E0FFF741FF2BE0FFF72AFDE8
:1029E00028E0FFF745FF25E0FFF74CFD22E0FFF769
:1029F0008DFE1FE0FFF72EFC1CE0FFF7C3FE19E081
:102A0000FFF776FE16E0FFF737FC13E0FFF7D8FE7E
:102A100010E0FFF715FE0DE0FFF740FC0AE0FFF7BE
:102A20005BFD07E0FFF74CFE04E0FFF765FD01E00A
:102A3000FFF702FC012001E00120404208BD982B75
:102A4000BED03EDC382B9BD01DDC1C2B00D187E791
:102A50000CDC0C2B00D178E702DC002BEAD0EBE792
:102A6000162B00D176E7182BE6D176E7282B00D17C
:102A70007CE702DC262BDFD175E72C2B00D179E730
:102A8000362BD9D179E7662B00D18AE70CDC4C2BA9
:102A900000D17CE702DC3C2BCED175E7562B00D170
:102AA00079E75C2BC8D179E76C2B00D17FE702DC9A
:102AB000682BC1D178E7762B00D17BE7882BBBD17F
:102AC0007BE7E62B00D19BE726DCC82B00D188E70B
:102AD0000CDCA82B00D17AE702DC9C2BACD173E78D
:102AE000B82B00D177E7BC2BA6D177E7D62B00D146
:102AF0007DE703DCCC2B00D09EE775E7D82B00D117
:102B000078E7DC2B00D097E777E7C046540C00103D
:102B1000645F0000B8040010F32B00D17CE70EDCEA
:102B2000EC2B00D172E703DCE82B00D084E76AE7E6
:102B3000F12B00D16DE7F22B00D07DE77AE7F62B81
:102B400000D16FE703DCF52B00D075E767E7F72BC3
:102B500000D16AE7F82B00D06EE769E738B5184C6A
:102B6000231C8C331868FFF729F9E26E154BA26617
:102B70000022E266DA6003229862251C10401C1CC9
:102B8000022809D090420AD0012802D0FFF788FE1F
:102B900007E0FFF7E5FA04E0FFF758F901E0FFF777
:102BA00007FB002807DDE368002B04D12B1C8C33C6
:102BB0001A6812181A6090352B681B182B6038BDE4
:102BC000B8040010540C0010034B0122DA660F22E7
:102BD0009A775A771A777047B804001010B5054CE9
:102BE0000549201C00F01AFFFFF7EEFF0123636682
:102BF00010BDC046B80400109C07000000B5074B8C
:102C000000201B680F2B08D1054B1A78824204D193
:102C10001868044B1840431E984100BD8400001002
:102C2000B804001000FFFF0038B5164B1A1C98328C
:102C30001268002A04D0144B1D6801231D4001E0D6
:102C400094331D68114CA3689D4202D16268002A2A
:102C500016D0002D02D1002B0AD111E00C4B1B68BD
:102C6000002B02D06168281C98470023636006E0AF
:102C7000074B1B68002B02D0281C291C9847A56015
:102C800038BDC046B804001098030010540C001062
:102C90009003001013B5002300930193244B1B688D
:102CA000002B02D0684601A998472249009B08786A
:102CB000214A00280CD0002B02D00223137035E0EB
:102CC0001378013BDBB21370002B2FD10B7009E09E
:102CD000002B0CD11378002B28D0013BDBB21370F2
:102CE000002B23D1154A1360154A13601EE01449C6
:102CF0000968581A44426041400010701148446904
:102D0000021C002C04D08B4202D10A2343610DE047
:102D100000290BD10A21516101999361D161084ABF
:102D20001360064B02221960034B1A7013BDC04694
:102D3000800300109C03001084030010880C001016
:102D4000840C0010540C001008B5FFF7A3FF08BD59
:102D500010B5094C20600948016009490A60094A18
:102D60001360094B029A1A60084B039A1A60084ACA
:102D7000084B1A6010BDC04690030010800300107D
:102D80008C030010880300107C03001084000010E6
:102D9000492D00007803001008B5084B084A19684F
:102DA00012688A1A1A6006D5FA2252001A60054B78
:102DB0001A6801321A60FFF737FF08BD880000105B
:102DC0007C03001098030010F7B50E1C0E21051CA3
:102DD000019200F023FE1A4B03240C279E420FDDC4
:102DE00009236B7301232B7328E0301C0A2100F0A8
:102DF00009FE301C29550A2100F0AEFD0134061CE5
:102E0000002E06D0E30F0022A7425341DBB29342CB
:102E1000EBD1019AA31A033B2B70621B2B1C01E020
:102E2000195D5973013BD1180229F9D10F231C1BDD
:102E3000002301E0013C2B55032CFBDCF7BDC04611
:102E4000FFC99A3B38B50C4B01221A700B4B02227A
:102E50001A700B4D0B4C08E01868884208D01B68AC
:102E60002360FFF799FFFFF715FF2B682168024ADF
:102E700010780028F0D138BD9C03001084030010A6
:102E80008803001094030010F7B51C4D9B235B00D2
:102E90000E1C1B4AE95C1B4BAC5CEB5C002902D0AE
:102EA0000F22144002E08021072449009A22520098
:102EB000AF5C154ACB1AAA5C3435BA1A80277F005A
:102EC000791A009107210C1B013210490194FEF779
:102ED000B0FE00230E4F33704124FF35301CFEF747
:102EE000F5FE2A786B783018D31A391C221C01346D
:102EF000FEF79FFE013D462CF0D1F7BDB80400104F
:102F0000370100002F01000035010000745F000050
:102F1000815F000070B5434B434C1A1C9432126819
:102F200090B0A061E161002A17D118280BD1C32904
:102F300009D13E4A12680F2A05D1181C38300E21DB
:102F4000162200F0DDF8A369182B04D1E369332BB6
:102F500001D100F07FF8FFF737FE0A23314D63619E
:102F6000334E01232B678C35FFF7F8FD2B68B342F6
:102F700016D006DC2F4A93420DD02F4A93423AD105
:102F80001DE02E4A934210D02D4A934220D02D4A64
:102F9000934230D10EE0254B1B680A2B2BD112E057
:102FA000224B1B680B2B26D10DE0204B1B680C2BF2
:102FB00021D108E01D4B1B680F2B1CD103E01B4BDC
:102FC0001B68102B17D1FFF72FFEFDF780F812E0DA
:102FD000164B1B680F2B0ED11B4C2368002B0AD0FD
:102FE000684608A9FFF750FF2368684608A9984774
:102FF0002B6827332B60154B1A68154B106819681E
:10300000884205D012681A60FFF7C6FEFFF742FE3D
:10301000044B1B6F002BA7D1FFF706FEFFF712FF33
:1030200010B070BDB8040010540C001084000010E3
:10303000130D0000070C00006A0C0000990D000041
:103040003E270000790D00008C030010880300105B
:103050009403001070B5254C23681D68FFF7F2FE3D
:1030600023681A689542FCD01E68FFF7ADFD204B1F
:103070000A22204C5A6118229A611522DA61231C17
:10308000903300221A60FFF79FFD2D36012323673E
:10309000FF36164C184D0AE0FFF760FD23682A68DA
:1030A0001968914203D01B682B60FFF775FE2368F7
:1030B0001B689E42F0D10F4C1820231C9033002136
:1030C0001D68FFF727FF0D4B281C196800F044FC12
:1030D0003834011C0422201CFFF776FE044B182212
:1030E0009A610022281CDA6170BDC0468803001076
:1030F000540C0010B8040010940300107C0300105E
:10310000F0B501240DE005780B1C254006E0C65CF7
:10311000ED0077083D43C554351C2540013BF6D5ED
:10312000013A002AEFDCF0BD30B504E0845C8D5C30
:1031300085548C5401329A42F8DD30BDF7B5099DB3
:103140000AAC2678089F2C7894461D1C002A0DD1C5
:1031500018E063465B5D4A5DD218131901920024A2
:10316000B34201DB9B1B012443550135BD42F0DD19
:103170000AE0CA5C12190024B24201DB921B01244E
:10318000C2540133BB42F4DD099B1C70F7BDF7B597
:10319000099E0AAC2778089D347800282FD0002992
:1031A0002AD01E1C9446002A0ED1013F18E0634627
:1031B0009B5D8A5DD21A131B00240192A34201DA9F
:1031C000DB19012483550136AE42F0DD37E0CA5CDD
:1031D000121B0024561C01D13A1C0124C254013395
:1031E000AB42F4DD2BE0D15C49420C1B211E01D027
:1031F000E1190124C1540133AB42F4DD1FE0002981
:103200001BD0181C002A06D10EE00E5C135C0130A6
:10321000F31A1C1BE40FA842F7DD10E0CA5C01336F
:10322000141B013462425441AB42F7DD07E0D15C2C
:10323000013349420C1B611E8C41AB42F7DD099AF8
:103240001470F7BD70B5049D01242C70141C002966
:1032500005D10BE0065D0A5D96420BD101349C421C
:10326000F8DD05E0815C002904D101329A42F9DDE4
:1032700000232B7070BD00B503E043185B78435406
:1032800001319142F9DB0023435400BD00B504E055
:103290008318013B1B788354013A8A42F8DC0023EF
:1032A000835400BDF0B5114B1A785B78825C1A40EC
:1032B00000D040220E4C0F49231C261C04C32C3680
:1032C00000221A6001240A1C123117785578C75D54
:1032D0003D4202D01F6827431F60023264008A42C9
:1032E000F3D10433B342EBD10020F0BD81010010D3
:1032F0001C0E0010CD00001030B512234B43334A92
:103300000131D3188A0051181A785C78825C144213
:1033100004D02F4A5F245218947054709A78DC7845
:10332000825C144204D02A4A7C245218533214700E
:103330001A795C79825C144204D0254A7C245218A4
:10334000A33214709A79DC79825C144207D0204C45
:103350005F226418251CA235A1342A7022701A7AC3
:103360005C7A825C144204D0194A7C245218A03240
:1033700014709A7ADC7A825C144204D0144A7C2459
:103380005218503214701A7B5C7B825C144207D056
:103390000F4C5F226418251C523551342A7022705C
:1033A0009A7BDC7B825C144204D0094A2E2452189A
:1033B000A43214701A7C5B7C825C134204D0044BF0
:1033C0005918F43127230B70002030BDCD000010B8
:1033D0008C0C0010F8B52D4C071C0025201C20215A
:1033E0004F22FEF753FC002D04D0221C7C233932DF
:1033F00023701370231C4F33002101351970503492
:10340000052DEBD1214B2D22181C38300270181CD1
:1034100037300270A1209A705A7040005F221A540F
:103420001B481A54A320400019541A4908784978B7
:10343000385C014204D0191C533152330A701A709F
:103440000024211C381C0134FFF756FF0A2CF8D148
:10345000114D124E00242B786A78FB5C1A4201D081
:10346000315905E03059FEF731FC0D49091A0A318E
:103470000C48043400F0DCFA0235242CEBD10A4964
:10348000084800F0D5FA0520F8BDC0468C0C0010A5
:1034900041010000810100108C000010A00000100C
:1034A00083010010CC0D0010895F0000F0B585B0DD
:1034B00001900027FDF784FA6A4C3E1C6A4A754267
:1034C000754113687D19012B05D168480D210C2227
:1034D000FDF714FB02E0002B00D1CDE0002303AA8E
:1034E000537023687F210B405C2B00D198E02ADCCD
:1034F000382B00D18EE013DC072B6AD006DC022BC0
:1035000000D193E0062B00D0B6E041E0212B00D1A2
:1035100084E0232B00D187E01C2B00D0ACE081E0BD
:103520004F2B4ED007DC3F2B62D0402B62D0392B83
:1035300000D0A1E064E0542B76D05B2B3FD0502B21
:1035400000D099E06AE0732B66D010DC662B3AD08D
:1035500005DC5E2B56D0622B00D08DE062E06F2B35
:103560003BD0712B52D06D2B00D085E02DE0792B14
:103570004AD006DC762B4BD0772B3DD0742B7BD1F9
:1035800046E07D2B23D07F2B25D07C2B74D135E0DA
:1035900031231370022E4BDD231C083B1B6819409E
:1035A000542908D0032E43D0231C0C3B1A687F23D8
:1035B0001340542B3CD14C2203AB1A7038E0322319
:1035C00035E0332333E0342331E035232FE0362355
:1035D0002DE037232BE0382329E039231370062E02
:1035E00026DD231F1B6819404723232920D11EE015
:1035F00030231CE02D231AE0412318E0422316E07B
:10360000432314E0442312E0452310E046230EE058
:1036100048230CE04C230AE0502308E0522306E044
:103620004F2304E0552302E04E2300E049231370AA
:10363000ADB203A8291C0022FDF7D6FA23681A06AA
:1036400005D5E91D89B20A480022FDF7CDFA2368A5
:10365000DA0572D50735A9B206480022FDF7C4FA8B
:103660006BE0C0461C0E0010900100101F3C0000D3
:10367000F4400000915F000023680122134206D04D
:10368000A818C0B2002107220223FDF717FA236809
:103690000222134205D0A81DC0B200210623FDF767
:1036A0000DFA236804210B4205D0A81DC0B20222E6
:1036B0000623FDF703FA236808210B4205D0681C96
:1036C000C0B207220223FDF7F9F92368DA0606D50E
:1036D000681CC0B2042102220623FDF7EFF923681B
:1036E0009A0606D5681CC0B2002102220623FDF707
:1036F000E5F923685A0606D5681CC0B204210722E2
:103700000223FDF7DBF923681A0607D5281C0930C8
:103710000222C0B20821131CFDF7D0F92368DA0594
:103720000BD5EDB2281C0930C0B20B210A35FDF7CC
:10373000AFF9E8B20A21FDF7ABF9013604340C37D2
:103740000B2E00D0BAE61B4803210622FDF7D6F95E
:10375000194D1A4E1A4F0024019A2B78D35C6A78BF
:103760001A4205D0A3009859395D0922FDF73CFAA9
:1037700001340235092CEFD1FFF740FA002814D0AC
:1037800006240321201C00F0E7F80321C5B2201C09
:1037900000F038F9281CC9B2FDF77AF9092C01D1DB
:1037A0000B24EEE701340E2CEBDDFDF713F905B029
:1037B000F0BDC0465C3B00008C000010940100107E
:1037C000C400001070B5041CFFF76CFD201CFFF74F
:1037D0006DFE0A4B1B78002B0ED0201CFFF7FAFD64
:1037E000074CC8235B00074EE518211C301C5034E1
:1037F000FEF714FAAC42F8D1002070BD9D03001012
:103800008C0C0010373B000000B589B000280ED0AA
:10381000FDF7A1F801A80921FEF7F2FA6846123077
:103820000A21FEF7EDFA01A8FFF7CCFF08E0FDF74B
:103830009AF8044B1B78002B02D00348FEF7EEF9F0
:1038400009B000BD9D030010935F000000B5FEE7C6
:1038500000B5FEE708B50A4B0A4A0B4903E01078A9
:103860000132187001338B42F9D3084B084900220A
:1038700001E01A7001338B42FBD3FCF73DFEFEE7FB
:1038800000000010EA5F0000B8010010B80100104D
:10389000480E001002B4714649084900095C49000D
:1038A0008E4402BC7047C04603B4714649084000CC
:1038B0004900095A49008E4403BC7047002934D09E
:1038C0000123002210B488422CD301242407A142F2
:1038D00004D2814202D209011B01F8E7E400A142AF
:1038E00004D2814202D249005B00F8E7884201D34A
:1038F000401A1A434C08A04202D3001B5C08224322
:103900008C08A04202D3001B9C082243CC08A04292
:1039100002D3001BDC082243002803D01B0901D07E
:103920000909E3E7101C10BC7047002801D00020F3
:10393000C04307B4024802A14018029003BDC0462C
:10394000D90000000029F0D003B5FFF7B9FF0EBC85
:103950004243891A1847C046002941D010B4041CBC
:103960004C40A44601230022002900D549420028EA
:1039700000D5404288422CD301242407A14204D21E
:10398000814202D209011B01F8E7E400A14204D2FE
:10399000814202D249005B00F8E7884201D3401A15
:1039A0001A434C08A04202D3001B5C0822438C0837
:1039B000A04202D3001B9C082243CC08A04202D3A1
:1039C000001BDC082243002803D01B0901D0090991
:1039D000E3E7101C6446002C00D5404210BC704741
:1039E000002806D003DB0020C043400801E080200F
:1039F000000607B4024802A14018029003BDC04669
:103A0000190000000029EBD003B5FFF7A7FF0EBC9B
:103A10004243891A1847C0467047C04600B500297E
:103A200005D000230139037001300029FAD100BD0F
:103A3000F8B5041CA30719D1231C04CB0F4D104E5D
:103A400050199043021C201C32420FD1181C0B4FFE
:103A500004CBD5199543354208D1181C074F04CB28
:103A6000D51995433542F1D000E001300378002BA1
:103A7000FBD1FEF734F9201CF8BDC046FFFEFEFE68
:103A8000808080802578000D0A413A200020202582
:103A9000633A20000D0A4D3A20002020473A2025A5
:103AA0003032780D0A0053455249414C20434F4E65
:103AB000534F4C450025732072656164790D0A00EF
:103AC000444D31364343000D0A4279652E2E2E0DAA
:103AD0000A004C43443A25303269202D20256900E4
:103AE0002573202573202025694D485A005638003B
:103AF000202025692E2530336956004241543A2052
:103B000025696D560D0A000D0A25303278202000F7
:103B100057616974696E6720666F722064617461B1
:103B20002E2E2E0D0A00426164206D6F64656C0DAF
:103B30000A00526561642025730D0A004F4B004650
:103B400041494C4544006F6E006F6666004C43442B
:103B50002064656275672025730D0A00000000006F
:103B60005C000C000C7C287C7C447C24104828548D
:103B700008000C00384400443800201008103810A9
:103B80008040001010100040002010083844380019
:103B90007C006454484454281C107C4C54243854F1
:103BA0002004740C28542808543800500080500019
:103BB000102844282828442810045408384C5C78DD
:103BC00014787C54283844447C44387C54447C1415
:103BD000043844347C107C007C0020403C7C106C19
:103BE0007C40407C087C7C047C7C447C7C140838D1
:103BF00044787C1468485424047C047C407C3C4019
:103C00003C7C207C6C106C1C601C64544C7C44001C
:103C1000081020447C00080408808080040800000C
:103C200007080400000000BF01BF010905000007EC
:103C3000000700070007130A00002000E400FC0052
:103C40003F00E700FC003F002700040F0800000CC5
:103C5000011E01FF03FF032201E201C2190D000052
:103C60000E001F0011019101FF007E00FC00FE010B
:103C700013011101F001E0140A0000EE00FF011130
:103C8000011101BF01EE00E0013001100105030048
:103C9000000F000F0A050000F800FE0307070104EB
:103CA0000B060000000001040707FE03F80F0800E0
:103CB0000000000A000E001F001F000E000A11097C
:103CC0000000100010001000FE00FE0010001000A8
:103CD00010080400000004800780030D0700001096
:103CE0000010001000100010001008040000000078
:103CF000800180010D07000C000FC003F0003C00A4
:103D00000F00030F080000FE00FF01010101010187
:103D100001FF01FE10080000000002010201FF0186
:103D2000FF0100010001100800008601C7016101C8
:103D3000210131011F010E010F08000082008301E3
:103D4000110111011101FF01EE11090000300038CD
:103D5000002C002600FF01FF012000200F080000BA
:103D600080009F011F0111011101F101E10F080005
:103D700000FC00FE010B0109010901F901F00F0827
:103D8000000001000100C101F1013D000F00030F1F
:103D9000080000EE00FF01110111011101FF01EE09
:103DA0000F0800001E003F0121012101A101FF00B9
:103DB0007E0804000000008C018C01080400000053
:103DC000048C078C0312090000200070005000D8FA
:103DD0000088008C0104010401110900004800481A
:103DE0000048004800480048004800481109000009
:103DF000040104018C018800D80050007000200DDF
:103E000007000002000300B101B9010F0006190DFF
:103E10000000F800FC010603FB06FD05050505058D
:103E2000FD05FF050601FC01F8120900008001F004
:103E3000017C004F004F007C00F00180010F080062
:103E400000FF01FF01110111011F01FE01E0110935
:103E500000007C00FE0083010101010101018301DA
:103E60008211090000FF01FF01010101010101832D
:103E700001FE007C10080000FF01FF01110111018B
:103E80001101110111010F080000FF01FF011100D4
:103E900011001100110001120900007C00FE0083D6
:103EA00001010121012101E301E20112090000FFEA
:103EB00001FF011000100010001000FF01FF010AB7
:103EC0000500000101FF01FF0101010B06000100D7
:103ED0000101010101FF01FF10080000FF01FF01C6
:103EE00038006C00C6008301010110080000FF01CA
:103EF000FF0100010001000100010001160B00009C
:103F0000FF01FF010F003C00F000F0003C000F003B
:103F1000FF01FF0112090000FF01FF010F001C005B
:103F20007000E001FF01FF01130A00007C00FE00A9
:103F300083010101010101018301FE007C0F0800E2
:103F400000FF01FF012100210021003F001E140A93
:103F500000007C00FE0083010101010101038307D1
:103F6000FE047C0412090000FF01FF012100210072
:103F70007100DF008E010001110900008E009F0119
:103F80001101110111011101F301E21109000001F8
:103F90000001000100FF01FF010100010001110902
:103FA00000007F00FF008001000100018001FF0090
:103FB0007F1109000007001F007800E001E0017890
:103FC000001F0007190D00000F007F00F001E00145
:103FD0007C001F001F007C00E001F0017F000F1239
:103FE0000900008301C7016C00380038006C00C76D
:103FF00001830111090000010007001E00F801F80B
:10400000011E00070001120900008101C1016101C8
:10401000310119010D010701030100070008000A21
:104020000100181110133831303378717073C8C122
:10403000C0C38881808384848782C5C4C7C27574E5
:10404000777235343732151417120207020802014D
:1040500000030109030402040205030500062024ED
:10406000282C383C4044484C4669726D7761726533
:104070002025735F56380D0A00252D313073202519
:10408000732573000D0A5479706520273C636F6DAA
:104090006D616E643E203F2720666F7220706172F2
:1040A000616D730D0A00557074696D652025757317
:1040B0000D0A003F0025730D0A0D0A00564F5941A5
:1040C000474552203E3E200025630048656C700045
:1040D0004E6F20706172616D73004B657920707254
:1040E000657373003C6B6579313E203C6B657932BA
:1040F0003E202E2E2E0044756D70206D656D6F7202
:1041000079006C004C6F6164206D656D6F72790091
:104110007400546F67676C6520646973706C6179B3
:10412000206F757470757420746F20636F6E736F79
:104130006C6500620052656164206261747465722E
:104140007920766F6C746167650000000080015013
:104150000080025000800350FC3F0150FC3F0250A1
:10416000FC3F0350E2A421299673065D6695C17851
:104170004AA7743638063C6875B5D4E3BE481221A8
:1041800089AFC95554733ED878B66102CCC20620B7
:104190008F6046575682A69D24CC06EA9B3E373652
:1041A0007F8D971E00130680EDC8FD7DDCB90D964E
:1041B000A2EFA34A4E48A56C70773F9FF4745E7BD4
:1041C0004D69D4E3B965F2361028698E740CE7891D
:1041D00099761DA2103F59A19A850202EDE0134283
:1041E000EC24E161AE2BF91CA370BE440D8711CD08
:1041F00072DCA86C138B426DEB7F8E393A659FEBB6
:104200005DA80D6B19E9ED01A09010117A77241AC1
:10421000B4585B098184EAD7B522ACF4515DD8BAB1
:1042200059C93A00596656B0972B4859C8D0A0AB27
:10423000BE6887CE80470A281CEB9A3813B24A859D
:1042400087D162031D2E468EC354EF07EDD0B18F88
:104250008D2C03583EDF6B95D592EE1E3A66771F84
:10426000496A76798600594345632B255759264874
:10427000000FD0E5520EED6277EC8F1A82851B009D
:104280000ECFBC97B9C33572B5B6A5712FFC0E0021
:10429000271828CA838E1FA7BF1FD89612491084DB
:1042A0001E8CCC4ED11DBF447D145C985BE2ED8921
:1042B000734E3C5F7F62648B47139BC81B8DD0D4C9
:1042C00053B5D489334ADC90BB70D512B4A85234AC
:1042D000260D8DB13CBF712C47F29A58CA6B64050C
:1042E0005AED354E8170A1241E94E7B0ECE184496B
:1042F00006B22483EFE53D97DFD3A56AD6080AF41A
:10430000F657B4F6E0745929A24B726F54B8DAE943
:104310004BA4715B6E11D5BE5249B036421ADD8591
:10432000A27B84622AC3FDD2CD851BD9DBB0262BAC
:1043300028BE495528136D4F608B77DDE986279796
:10434000D0B7F725DF147B82F5113967766ED08BF5
:104350007C417004DD6F57ADFD536F8546BB92EA1B
:10436000E7469F83AF568F99BA871590005255DC68
:104370003F6A2FD40B6A49465CA41C6E4AAD85ADDA
:10438000C7DA5097F2D5F0CE910DA4FC25508BFDE5
:10439000C4A9619050E81BEAE8DC6A9E305E54EEE6
:1043A0002573F075D2983B5936A79B18C521C0AD2F
:1043B00059C65B03F655B1F8E9F53127416951FD5E
:1043C000C1785EC31FC561A94D05E68D0EC89C98D6
:1043D00041A7918188AC7623145FFC1BC69D17A969
:1043E000FAA0602004EB8DCE165A93706CBAD005FB
:1043F0000F0D6757012AD685C6AB44917E1502BEC4
:10440000D0269E5B9B350E8ABF039F0484CE6483B7
:1044100011F66F9BE0D3320BC4A513BAC4D5332178
:10442000032BEC144DA050879180C31B123B817469
:10443000A462210D35E77A2EF0E67600FD5DCD020F
:10444000776DB000F610EBAEC2AB04CD642537BF7C
:104450008F0EFB9634D15482D6933714FC0438A9BE
:10446000F5139D201C99664DB5543552CA5EC5762C
:10447000289FF1DD74BEE5CEA305BE108A1ACD20BB
:10448000E00A565404F23F4D54E21D42672C14A931
:104490005A4FB3BBDC1BC5E69A5D6F7AA0EB853D36
:1044A0001F92EEE531A6E8D82036ED6946A701C790
:1044B0008F82BBC6DE7AD63954F8F8D1DF619944D1
:1044C0006D1310143CAEDCD9164E40CC85E2FC27AF
:1044D000B68DAF2997933A7D9C348E65F10E4A379D
:1044E000B7538FC97501E49D7850B292B39EDB84B7
:1044F00000726B139C87AD8C24862BE6B97F83D02A
:104500008C5D215092413C6E4120054BCFD662B369
:1045100051109ABEC50372FD89DC5E5B4503598765
:10452000C1D5001AF2193974D51AB70126599089E4
:1045300084B871C9F1E2E7ADABFFBD96D2A4D81F34
:10454000CD1FF9773493EF646A22FD409416F2216F
:104550009E5FE6D4BDA92C2CC3446A1B93BAB0D489
:10456000FDAA3367B35E0A856E275ACA92FB2F7A7B
:10457000FA0EE9B1801B071A14B2320E3EE23A403D
:10458000A530553B66BA810C93725FFA14E997A97E
:104590004D65F12EED65DA07CDC8B1BF5E1D85957D
:1045A000BF6E51B1504CDEC998620CF3ABD7933556
:1045B000D0E8904F46A207BB7D214CC0CF4BEC7694
:1045C000E0DD202F8C85451B4A334465989CF6D846
:1045D000824BBE3683992EE7D4C50358600C2CA7B6
:1045E0007B9B28F626EEC79AB1318800D459A804DF
:1045F0005B7D4AB0CBBDED4EAADB7994FAD9E7EBEF
:104600001272895B8FB91DC3D182D2B9603CF51B90
:1046100081456921B781294A908D46ADBC88ED91CD
:1046200088BB18CF80F943E5C8862F9B407B0F9746
:10463000F2E30C338C48FB1672EF8B5F0287AB8A78
:104640000674E208EF0EE578B9E2FB048B052D371E
:10465000A4B5E4F86B24F26E87AB80B786FF854182
:10466000BFCD16DD3A4142E36C0427FB552E1BEB10
:10467000EADA55220F998D92417046B6F9852DC11F
:10468000D1739152CE3387D13EB29D0125FE2DCB01
:10469000B50B4DDDB47EB76C511163308929584A92
:1046A0003BAC1F6B9F7E2E0D2D045A45C9BD87D98B
:1046B000FD9CCB1E2230FE6AAA5C0084770BC135BC
:1046C00041F173835EB2E45D3AD83BBBEF1FE5E195
:1046D0006D10406AF8073C392BCB625FA2762AD96D
:1046E00087171B5B4263E119FCF1FA9C0935911AAB
:1046F000C5A0519CD41690717DE2593C0407DB5152
:104700001122A4020C608F8FD0950D088E969CE22A
:104710002D33B8425DF3CB02D84F9B539E1F14EF4D
:104720006E3F70F7F55C4EE713B9070D86209F8E3C
:104730005ECB8B8C6BEE579EAB34966D6995BBD37D
:104740007E683D1043B5FEFBBBFE9161296411728A
:10475000FA10EFFDC94F563D20AFDB1AF97B6D0013
:10476000EF84F29D01756ED4FBA86EA39954575E39
:10477000A09DF29CEC0024FECD2DAB7199CFFEFDE7
:10478000DD369C91DCDA554A1E5A8A82EA8A9B867B
:10479000015D3DD672AB395B179987242954A26A13
:1047A000968B04674C71548AFE5B05234426C2A194
:1047B000850BA4DA0B7B660CF31260035792F73F6C
:1047C00043067CCF715E45CEDBFC9D219E9C41E87B
:1047D0004AA9EA9870877F9B1C323D83B17C8FD6B3
:1047E0004842FF637200778BC027FF4141020B3CB8
:1047F000B77B528E4031EB60A9D7E74378771EE252
:10480000ABD4DC5B1CFC9483DB431F7F2F914E9E5B
:10481000C3CEC789170E901CFEB1619562F2F12AD2
:104820003DC58AB42827822E1992C94E871275B3C6
:1048300002A5EBEA568FA1A70A3E06D2EB5BDA9FF0
:10484000EE2A325A9D1B69A50508CFBB67C45726BF
:104850000F02476F6563AC3A8D2DA43BE283780964
:10486000B924E2F5BE76D5D3ED1CCD6914FAF40275
:10487000FBF6B86930A9BC4A7287074E5DB10AE5FC
:10488000977B9C1AFDF0AA9BD36F94CE0459D67DDA
:10489000CE0D7FA94E066723F1CFB5C408832CCE79
:1048A000021A4006A600620D2D7CECA5C689595E51
:1048B000A3CB0A7C82ED9CD6716B51830ADA768396
:1048C00014C74DD3333FC1A6298DF1CA3F8D690668
:1048D000976C48AD8595D7298F2A6F62BE40B02E60
:1048E000A7F085C2C3C374A4D7EE750BC77E2CD1C5
:1048F000F455A4F42C7F8260A8DDCC24CEEAC361F9
:10490000320DF2A17CDD388EBCCA37BAE6CBD0B00E
:104910002F99F7CCA2B4694A98B7047D8AED207D1F
:1049200079F48A218911883B1FAD9437B3C1DECB5E
:10493000824FC5EC817F2FC5D3E9CFF683426387D1
:104940006E16B87996F547721E90D6B86F950CB66C
:10495000EC6FE50C8C611152D503C588686B36EAA3
:10496000D717EB0C0745654D0BDB70952478F7FBEB
:1049700056A915C43B56BD9B6F0374B4BDBED0157C
:104980005FE669DD95F668B58BCA115AE15FF28979
:1049900092CF22FB53A57B214F2D92759F6098E902
:1049A000B62EC278120F193A156C1EF893FEDA2350
:1049B0007770B7D2D50D91B5088C2FB4F16EF65241
:1049C00079A9419B28DC27671A009DC905FF1F5361
:1049D00007BAC8C1499FF6EB6C5DD7AA3FAD03E7A4
:1049E000CD6D4B112E227362DC215DD90047267CF0
:1049F000A5876DDA75BD7A4520542BCE370DA736C5
:104A00000214893D84A7602E2BAE7D5A4ACF92179F
:104A10003974B32783080BA340B5912784FC1B830B
:104A200025B8503AC9F7E3600D865E59092002D7D0
:104A3000B63016DD2FBF86936A1FE349C65F4C6808
:104A4000F75AD913838BBF3397ECF05A44D11F1E0A
:104A5000D397B1B0A09CCEDF08F6648FACF74410BA
:104A600091BBABA80FF605D90E116584AE199FC690
:104A7000376566CE21C38CE972AA0A36B8A238FD22
:104A8000BBC44A2ADE75B22C4E40144D076EF32F7C
:104A90007FC7897F5EF9B7C663A074030753D0CC84
:104AA000FAEAE5E26A497FDD96D85109C29416DA3E
:104AB0005ACB2ABAE6278591BD0D6148FE400A69A6
:104AC0004E656D6FCF764AB569636022DE4868F740
:104AD000476009D9A4EE32433A0C0164650AAC8BF5
:104AE000444E2144A0CFF3E527D908498935959054
:104AF00088C33CA15A58C408FC92D8FC0B45C50594
:104B000033A75CBADD1B1F1984ADFEA2D42A67ADA2
:104B1000DB3EA385BE4A87E8269335CF9F848C0F62
:104B200046C26AA306D078493AE13F232405584D8E
:104B30000E0A916C7F59B0694A12ED8AB1E4A3362E
:104B4000D2D7F876A71174D644365E5BC82F12F020
:104B500089BB8E10616A2E261EB82909ECF3FD95DB
:104B6000B468B31AEB5253A6DF41CA9A77C4E6ADD4
:104B700074D44B1E3425E0B0BD5EBF148F327C85EB
:104B8000B6D51343C202D60A13BEB0EAA8EB7A2CFC
:104B9000EE7E2EBBCBEB64ECBF79CD809EFAA5E90F
:104BA0003D08379390981785063A0029ED35813AEC
:104BB0009EF4AD826C22DEEFA8879E468B22891080
:104BC00081C26A5082565A2D1FBAD7567658582A33
:104BD000F7CA4F2BCC902B19819A8FD524259C583E
:104BE000C6E20F3A270AA30875C037193E8AE10EBC
:104BF000A3A046AEA9113C1FAEA961064A83B8A482
:104C00009529D24FC04C547587432943E658040870
:104C10007E58D9A96CA3B7BDA678C70BB5BA2178C1
:104C20006A432462E19B2E6293B78B43B597A70B2F
:104C3000D50A3705E0726E57787C2EF79D9661098C
:104C4000989E74286B24043669CC887053ADC5F9DE
:104C5000F45E5747E61E5C525BBE448AC5318258FB
:104C6000D2429D4D631462354FF176D23C583A776B
:104C7000DF55EA17AB74D3CA1BC9E47D36F75F383A
:104C8000BE0F94164F9B34C2C5CB4B33DB83ED4133
:104C9000E10469BB2B31D980008B7E13BBA7739CC9
:104CA0005C2F2C3C8F651BC68EB087CBEFABA96603
:104CB000C41E58FEE49847AC16722CAE2C7723B174
:104CC00071839D364F545F3DFC6E42F142EFA80B5D
:104CD000024486767E5FE6EBC6ACB4C941E2E806E4
:104CE00000BB38941B40294368A3514902CF811B64
:104CF00053294F442173DADA8B44750866B0E0AC6F
:104D000076BDE2FC5A8B7C6EFD16AA422F7257E2EA
:104D10002171DD0F09D0E64AFDE6DB162FB56016DE
:104D2000F4CAC1BE2BE7F7E68A84B39214B8136ABB
:104D30004855A94E935F9719403AF846053CCA1763
:104D40003DC2DA6F5ABEEBABD25DA0861F66E85754
:104D500064026B9144F01EEC6A06B238829E9A554A
:104D6000C9A5C7B90773CEEF83DDB4715F8E14BFD9
:104D700025EC7D6875E6D3F202C7FA05BDFA2E3739
:104D8000C047D3A7181DDA67B79AAD4D69389E2979
:104D9000BF0E4AA039FAEEB84A72845A70045AE932
:104DA000C3B65277729EEDA733F2C3829A1ABFA29E
:104DB0000C5E702D4AFBC10A5E21B255FFEB5F5FAE
:104DC0005E0DB541FC421BD946A9CBFB5844611E80
:104DD000722328A2A979EB3EC3916A311FA405680A
:104DE000CA8BB075A53272FAE78D37FEC61209C8B4
:104DF0004858A90ABACA2BBDE411E96872AE3CF65C
:104E0000FC41EE5ED9F82AAD0066F2B0D91A64878B
:104E10007600F18038921BF7139C422E7C8E9649C7
:104E2000FCED51A8DB07ED7A621931FA9B2D182FA2
:104E30005EE99328FCE47896EA4F24C0E7B8F2B123
:104E40003DF0AD48525CADB6646CCCC454A5B7839C
:104E5000897FD3EDBF4397E8EC592F4ECED835CE9E
:104E6000DAEE80CD10A1B943CA33B60FB3F74CD7F1
:104E70006286379BFB43266796466228D08D2AB60A
:104E8000EE28687726E2E2A243C182E4F25C19DEF2
:104E900082BC97824171981F9422CF5177D1BAD2A8
:104EA000DB19508C324E917720DC479C4052A5FE96
:104EB0000A492C64C2DC32CC889F89DAAC20AA6E05
:104EC000D753F7B8742C0921842EF2DBB0F50ADC35
:104ED000FCB4E3BED1CCF490B670DDEBA9E0365D56
:104EE00018B723BFD90BA2CF72C26AD95B13570878
:104EF0002762B85F730DA6186E8A71F8DDB0F49161
:104F00009CE16C3EFA068F4099F765F531689B4F3E
:104F1000F1DD74161BE07B9D5A8577DB12F3FB8372
:104F20003FC029BF47448E64FAAD1610EBD06974B8
:104F30006D0EBC4431A16A9D6BF149BED5F19B6AEF
:104F40000DBB702B2BB099BE291BC98DCE51738F11
:104F50003D20F3930EA749A521DB14FFC020DC45BB
:104F60000C0516C7718654191BB8F6DC89274289CF
:104F7000F123C29F63EA925DCA74DA7027821D949E
:104F800024DC59BABC3D7CF2AA231312C75A003F55
:104F90004261C29D4F123F0A1C7DCB4E4457BA6EF0
:104FA000AB40323D31F2BF0F95520047CFB80A6097
:104FB0007594D0036E35D9B5CB9E865423A9C2040F
:104FC000C4F1429CD5DB6781A257ADC6A7D2C93ACE
:104FD00062DE65640A6B9A4E9C3FFE469C448328C1
:104FE000BC478CB394329E03045DA583D44119E879
:104FF000715F2196AD47DF087DC9E2E854D62FE600
:10500000C07E1A847935176F58858541C62EF8D52C
:10501000931578839A67E64169DCF0CE5C6C216079
:10502000648C2F497876F412D51ACDBADFB71145C2
:10503000DFDDCBFE4E1FB161CA0C34D8A927719AAF
:10504000CAE1ACBA145E1C9AEEB3081D02F232D863
:105050002200F3BEEC40EA67C3585AF8275573AEF6
:1050600036B2E47BF93CC78ACEAC7DAB5A5997CEB9
:1050700079FB2E85EF112E13DC6529CC918DF5334C
:1050800025012F0D4BB75955EAA19A219A1E71920D
:105090005C54A69F31D51FD92FD4FD358892583343
:1050A000AF0C4083AAB676EE2E03E12BC746C79716
:1050B000EFD186AF5842041ECFDAB958857416F086
:1050C0009103A297CF269C77D3458C06E44F604D81
:1050D000D393AA4DCEC90D184A4353A7C784B7210D
:1050E000CC0438A3CF4BBAB6D952A3662A4939E1CA
:1050F000AF7AB18D8F1E95BE546E91CDEDD9D8404B
:10510000A2C76932D0FEFCF29CEC8B9C2F1E1A6366
:10511000FD8BD75E21D838E20136D9D4CCB0E73F39
:10512000AB72D634B5C3A20B9D54F39FB356379ED2
:10513000B4053703CA283C09593EDE0CDEACEA57F9
:105140001647434D241ACAB6B3BC7E6AC178EA0C2E
:10515000D6BB7BEF5633988260DF4B352EC1F931D9
:105160001EBFF769F237938E9E70ED2E60A3AB439E
:10517000488AFAD0FA2B7D98E910595B96AE6EEA10
:105180005C9A1C7EA5783BFCF88DE43FE4CEA90731
:10519000C08AC187A214608093FDC2E997765E52EF
:1051A00034FFDF24316384C7A8C25D92A2C36E229C
:1051B000156CC55610640B4895BE02CB39A04F73D1
:1051C0004B82E473D8BDEBA5D6366945C66F0F890F
:1051D0008B14B4E2946326D00C5F54B6833D7ECC2E
:1051E000E90E5449D61DBEE9E645BA1F2B76B4F840
:1051F000BB13181F7E5C46508E3F8CAE956865D001
:10520000F8F16FB2C1A0CE33CB0B6D70D1284D0930
:10521000A518013AB39B0C4ECFB834005E060808BF
:105220006E1D699AD65D7996B57FE3583758197423
:105230006233373F87764ECB5D529060BCEB45E2E0
:105240000142E4F06BD588E2FAE15D3D4C6B010769
:105250005D3FD9B49DE288EE45F3A8004F707BB264
:105260005BF70B99B1DFBE25712BE589087ED5BDB3
:1052700017EB65EB6434CA764B06754E11C7A35B1A
:1052800025EA937A388BB5F35E615BEF45B38A69A3
:1052900060B22931D969A5707DF2568EEA91AE09C6
:1052A000AB42223241F338CE01475D62E24BE17DF1
:1052B0006FF6FDDA896F905F86A2BB88CFD35E530D
:1052C0008504E6B45E61984E930E1D1D40DCE5DA60
:1052D000BC2D65C2400308C7750055E1285BEF513E
:1052E0004DB125CC8A22F5782936F7C0EDEA4DE399
:1052F0006B2D0F4C1D1C72573D7B651926244200F7
:1053000014296138F601200C943B501325C4A69053
:105310008EB1F1B64CD01970B4F349FBD77F02ECD3
:10532000E7AADDD0D1C2EA6CC58CB2FAB7C769F77B
:105330008C2E4F7CD1C6AB2E233C84F950B13A2D34
:1053400025709A0D318299629542BBF78FE7C011A3
:10535000BC096D7AE63021276E7E3F13C4C6E11486
:10536000983A42E6FF0E6B3B214E43AFF6AEC2A326
:10537000ADC7D5AA8FE51433DE1C2D512F75EA1C5D
:10538000C570B8F62FC04A94C1EF249475A6FA14DC
:105390009410C774555EE5FC0F4B76ECF265817B8B
:1053A00034E0D62EBB3136FFAE5FB348DE0C1FC9EA
:1053B00099596B640F3A1865869E86156503C51169
:1053C000F997F5064159A58BED545589A1D9846605
:1053D0005160A923F4E0E0EB11FF59030B4F8D2D31
:1053E000B200DE85D8F8B9373970D468023CD1C82C
:1053F000E4049ABAB383656A1E532A8E093327FEE2
:10540000350EA53A488D91C7E06FEAA3F28E05E606
:10541000F2AC47538A06974228B922DE2BB4978A0A
:10542000B92F27C60C62B22F29FDC920FED0ED3955
:10543000137886619B4F8E23B848771E66C2D7F1DA
:105440003663620EB7B4FFFAB20B42CC3EC46F4E65
:1054500021EFE2ADF6BEC8DE6F8C4AC9ED2A0CB86A
:10546000ED51398C55FB8B13EC1AAB03AAA46D617B
:105470004FFD41C421169CB87D98E795C764575DE0
:10548000B5988E838607EDA1BD14E484BEB289EB86
:105490002E98B11FB2B3FCF213469A156DDD3E385B
:1054A0001DB1E96184893B3B715EA6C985BBE604F9
:1054B000B14B2C8552F5F109F00E46682D22E7D844
:1054C000E87B33157D5BEA514932F2E2CE1683392F
:1054D00097373C78A6983A381DB824059D583E4326
:1054E000E73A12D1A9A845CB9E3FCC315D2E5BA2F5
:1054F0009649E802F0CD2A17827BE2E0CC46375B82
:105500001CA38F8516765E319684F1D7A61BEC4FCF
:10551000906EADD64D3BFA796CB35019D109074363
:10552000EF78E01B07D176E6EAB35E4EFD1D87619A
:10553000D964353B03D43CC26642F215CF27D63F2F
:105540009074B261F4E3EB846D9C3E314EC9D4A6F5
:10555000258B4FE69B19DA44E76003452382451407
:1055600048D95260C939A743565D79F720B2C2E7DE
:10557000D01AAE1EFCB5822A9AB3EF0970158A5C68
:10558000628EF5D3DD146E9FD2B6C4536533E9271E
:1055900021284D72623F2D81E3974A2EEF34E4CEED
:1055A0000974D102999497256E19B440B3147C2CD8
:1055B000F346CE098882A9310277E7CC3DE4EAA31D
:1055C000DE3681ABDC820432F6FBC5D5171D2B4BD2
:1055D000D5B78D6F7C83F2C442001372E91FEC5083
:1055E000F06FB8AA5AA900FDF54BDBFE37871C8E79
:1055F0000051718AC97526122558B2840F599C92A0
:1056000035366F1008A0B32EC633AD7AF315A73226
:10561000F873D9F5F3A1F8E5C3EEE9658728731FA0
:10562000819504CF3261CFBBB65A948C80A15623AA
:10563000C96AD455FAC3EEFA15A5FA87BF20DF5719
:1056400080FC255314793884CC9B131946BACD219C
:1056500007864E853F9727B273873ACD21255CAFE9
:10566000632662CDDDC3C1170EE4EC22DC485D3653
:10567000EAA4060DB79D75F952E48E132D94EB2A1A
:10568000A2E99193C14F6BA866502353A1F29D925A
:105690004F1C88129CD29C1B3D9E93044E0A9A9CE0
:1056A000B18483FCD974ECEF72CDB4520B229A41D1
:1056B000CD35E70846B8B8CEAFBA1950B3210FCEF2
:1056C000CF929676847D3AF58DB77E7C0063DA16AC
:1056D0005F55B7CA492FB63FD8150B1D5D0B4D6EF0
:1056E000881EEA776508965DBD84AFC7C981233CF3
:1056F000D7C7EDDBF30295963C1AB6D3D4695C515B
:1057000018AADEB0695F46D976E562C5D1A87A8F5E
:10571000D1746D09144D91FDEEC0DBF62A4C9A6DE3
:10572000217C55E33E26BD98BDC9AB4D9EB71E0FEB
:10573000E01D052E2FB9C5B0F372A7EC0B112CDCC0
:1057400043B3F3DCE2B46C8957578A8173C3537B4C
:10575000430E1FA22C80F4BD49AE6CBF00B50E7F76
:10576000EB86FC004A43ED5E5018A35E82E3338E65
:105770009C715CC422410193FA0C7431C49201D92A
:105780009AD413A1F5E4028AC0805FF520E9C3BA78
:105790000F3A5F25A83DAA0D6FFD24F2200048F5C1
:1057A00053C037C622943A3A22420007D74A4D9A4C
:1057B000A48AABD7CE7A068943717D6149E344BCA4
:1057C000AF3FA8554E1BF4C9C652DEBB71DFEE0FCA
:1057D000F9C5B58A486570565B3139A65BDAD9FEE2
:1057E0006FDFBF2162E8AEE8D161F14DF57F079E22
:1057F00074DBA5A31329017E6237F2AA49156F88CD
:105800002282FFD9C65E2150228F2B3800FFFF393C
:105810009ED6F921AD58928FDF338E49BD0CA5BFBE
:10582000A30BF7FDBC4C93D7288FADFE73C8D828C7
:10583000B358F5DDFCF897C7E62A2AEBBE4982E1AA
:10584000B1505E4E0F1DBE3A8A45D0DC29EAF060A9
:1058500063091A24E25FF4298889A25512D446917B
:105860000DCF6A9CDE2A347231DB457970A6FBDCF1
:105870002D32220E6415EFB6A3E1F1D0F90CD29FC0
:105880008E26EFC612682CEAB253A939B5F94C77C7
:105890004D782F1A59A6E9BF81A44795ADF0AE5FA8
:1058A0000AEFADC9B6E95A09097C82FBA430C102EE
:1058B000E759B290DE9781BF89292E99AD4F498271
:1058C000A8376CDB3F54429AD8F374BFDA252ED444
:1058D000CD69C799A5A2354A40A2183406CC6C916F
:1058E000C2436407EB05F7F67CC4503DE4E937B2E8
:1058F000AB2B4C731B3F76A3663CB7D22E916DB594
:105900003FE1D5D3043A65CD9E010CC795CA8C649E
:105910003DCF2DC5D050F3C213C0D5F112D8988613
:105920005246BD02C988D9666609C8A19FB651EA28
:1059300056995BBB685EF90C789A849683261A9810
:1059400049525068248DA6DEFF730F7BB67ED83790
:105950002675A8DACA6AA867FF62550B9AEC6E0230
:10596000C1E52CFCE73EDCAFFD0740898046D1F461
:10597000FC2A915547C90EFBE817A59A8C5B42A6F5
:10598000D84185D43D558C416A497763D682CEACE7
:10599000C372070C677FA79E5945E35DE2BA1AA65A
:1059A000A073B2A8B71775CF1A6C566CE4D28158A1
:1059B0000DCA10732BAC0A75BBD2EB0A015AA02892
:1059C0001A8571E1F65661E4C8912A74E50295BC26
:1059D000F6D16E7C3308ED71BB9F4AB40F437A0950
:1059E0004F6C28B41031C898D6D73F25C997ADCC95
:1059F000D7261DEB3A8B4D728EE4958AC05BF4DF9F
:105A00005ECE12362F83D33C5D82FDFD7F12DBC25A
:105A1000E2C76CD1A318FE999552BFFEC195333EE3
:105A20007F9951A6F4FB834809603EDF2B699C6A8D
:105A30002AF5631CCF23627860D037EFCAD33AEBE4
:105A4000AD57669AA07742573D62A0DD94BFE2E968
:105A5000DC9F1C299727C8267EA21292E15729763F
:105A60008D51F8A47D037A5AE6DA33860A926BEEFA
:105A70000EC2D1EF0F82EE2DC6180AE9543F97C32C
:105A80003C87C943575BE4D456A6066081D8369F4D
:105A9000288F9965CCC53C49AC1C1BEFD390A190D5
:105AA0003308485317E4196F21B7B49DB3F541F893
:105AB000892CFF7944CC842AFAA207BB64BB2888CE
:105AC000CFBABF991BDBAD55FE248E1D4B68AA33A0
:105AD0004396D21F3F8FCAC43529CCB149C0F708BD
:105AE0002474142234512EDB2A5D65F8DA5881A81B
:105AF000CB1C3CB61A13FE9D0F3EEC6F38D667E404
:105B000024110F4B5164CD2B1824675D60B9828A34
:105B10008D671BDCA7E914A650AA08F168C8544297
:105B2000B8B8E9A3D984209D5ADCA9D34106409492
:105B3000F20DB16D514CFA0763A8563FECD596A80B
:105B400039574D23398141B28658E59C68A51AAD75
:105B50004ADFF1AC78AB6B8D6C8E14E34B70340282
:105B6000ED273EB0C506D67E845B5AC2AA25BD2B62
:105B7000746502C6045E87E82F5A2C8B45162E4AA0
:105B800013F55D7C4B457A0A3883254CB0B0A3C829
:105B90002FEFA37BB2F38AC440AB51C5275B606192
:105BA0006A2BC4C1212091BA49263F92658E75ABFC
:105BB00023CCE9BCDFB1431622CE83AFD95D30627E
:105BC0001BCBA6594035E7C897FF22806A28545B53
:105BD00041EB053C47FBD6740CA99D4087849B385C
:105BE00026748D636681F852BFE055A92D4BA53C04
:105BF00015A1C32DE0658FBD53846400ABDCFBC6EB
:105C0000F50951C29710EEDEB27A97120A48C26FB8
:105C10003EA57B7530E41E0AFB16F689622231DC54
:105C2000C7015AC9D87C228C57B04749BDAF95BA35
:105C3000EF3AE450F37C2345980B7EE7E0B612651B
:105C4000D74C0F3DCC1A7933B2FE85B3295727BC08
:105C5000E5FB391582293832B89117C7E15AFBBEE6
:105C6000990F3772688AE2B6958E3E41115525C06C
:105C7000632AA28B362AFE5F9FC900F5DB9FBC7C9E
:105C80002AA4A7212EF546FEEF27F26A4C420A0904
:105C90002BD8592351EAC18A7C51CBEB6D23BFC26B
:105CA0008CFB26BE9D0C6C662C92775BBF01C0D628
:105CB000F9E0793F7683DE18195B64EF3E484BDCF0
:105CC000F74894211C9B76BE1DBC334A3561E9C55B
:105CD000A4E97C23AFAD5DA6352AA918F113BA4516
:105CE000EFD89288425304FA28609D0182CD7992C0
:105CF0002C63A1E20EEB0F2624D7FD3E606B400A19
:105D0000228D431F7688552EA934D6252402587F2C
:105D100033DAA778A0CCEEAFD522BE002473FCA363
:105D2000C3857B815501A05E96EB6DF4DDBFD56226
:105D3000CC018F5D5AE042122DBA0CFCB715225AE5
:105D4000D79101717827542552455ABE6ECCE98807
:105D50006C0A6BA75275A5B5BE676880950BDF2BE3
:105D6000063910698BE6831221EC31441FE219F2E7
:105D7000DA7F2D408F240C45998771C0D82227ECFB
:105D8000C06A965465E7E2CFBF98E493D6B8C18D58
:105D90005F993A966FAB7B65D8FA96F617DF0546A2
:105DA000331C9E849A567D06F21E587336B8F38CC7
:105DB0001E29258D31D67B4569C4BA758EEF365FB5
:105DC000193E5A2FBF36B3AA38CB13285210930D61
:105DD0007C1AA2FB4538C3F01A2EDD689B1773129C
:105DE0006D84BD99F19D4FC8AE1289910CAFBE83F1
:105DF0005F9C579D340B4A4CE0983DD67323C0D727
:105E000029C1598D9D4E14F2EC21902F0325D3F317
:105E1000B32E584246CF9D79CECAE51ABF9C538017
:105E2000F8F147040247F5E82940AEA5BC793A9F4E
:105E30005B82EB3508469CC8EC765CCBD1011FB584
:105E400010B6A94295B85A3B927B2EC15470E5D347
:105E5000C774184D065818029EF3BCC3DDAB8118F9
:105E60002EB7324D41609A22B4758C5A12C0DED7DB
:105E7000D32AB59DC7F3D08602D7FB4699095F5A4E
:105E8000F0A63342CB16226D19C680043D43BA7D7D
:105E900044910CA7585951B06B491A290E1580D757
:105EA0001C7518FD3966FE1D60D122D842E0080D30
:105EB0001D123B75F8C613291236B28D21BB831310
:105EC0007715943705D15816AB08DF8479630F2511
:105ED000ECC611ECD86E099E06F2514F62838DEB31
:105EE000C035CF203E68332F7B3527C1E728526D60
:105EF00000DA2C2223B4EDBD587298F629AD4CF38C
:105F0000458845DF2AF4FE1F45D6A09057B91554A1
:105F100021282836001D583D8CE102E3A35578BCAA
:105F200095E7A0C3A723C0622334B2B6E5ACE496DC
:105F3000C5427C2FB9F703105E50DA741AFDB665BE
:105F4000D0046996A859E5B760264D59628B76361C
:105F50005C2B30EEB3B4534049C4ABEFF19CD4CDCD
:105F6000E223282F0304050A08060BFF0209070D88
:105F7000010C00FF2025692025692025692D256950
:105F800000202025633A256900202020205F5F7CC7
:105F9000002C0044697370206F66660D0A0055532B
:105FA00045520046004700424547494E0052414491
:105FB00000442E4D59005052474D00555345522034
:105FC0002020006620200067202000424547494EDF
:105FD00020202020200052414420202000442E4D2B
:105FE0005920202000432020200005000000FFFF52
:105FF000FFFF4D000000B3400000000000003D1016
:106000000000CB400000D0400000CE400000FF0068
:10601000000001080000DA400000E4400000824077
:1060200000000000000021060000F6400000D04003
:1060300000000241000000000000C1060000044111
:106040000000D0400000104100000000000059088E
:10605000000012410000D040000033410000000069
:106060000000E905000035410000D04000000F00AD
:106070000000F40100000401030102010104110405
:106080000F041704160118010000BB5F0000C35F76
:106090000000C75F0000CB5F0000A55F0000D65F77
:1060A0000000DD5F0000E55F0000B65F0000001744
:1060B0001B243E425369750502050804080B0804B9
:1060C000040501050409080904060807020602047C
:1060D00002060106040701030803040C080D020C64
:1060E0000203020C010C040D010D080D0408020846
:1060F0000807080202070408010804090209010A46
:10610000080B020A0201080A010A040B0102080234
:1061100004100811021002110810011004110112DC
:106120000212011302130812080F081204130113BC
:106130000414021401150215081408170814041594
:106140000115041702170119081A0219021602197B
:106150000119041A01160816041B021B081A081854
:10616000021A041B011B04180818040B0420202029
:1061700020202020202020000000010000009E5F41
:106180000000A35F0000A55F0000A75F0000A55FFF
:106190000000AD5F0000B15F0000C53A0000B65FCF
:0261A0000000FD
:00000001FF
